:020000040000FA
:1000000064002500170A0A0281000307090AEA01B1
:100010000008EA01E8030D0AA902EC03100AAD0288
:10002000EF03130AB002F103160AB2020008000C33
:1000300026000F0C0200F80C0600070C24006000DC
:10004000A40243071F0A610086072A0A26062A0A15
:1000500007052B0A070403090B06340A0607340AAE
:10006000680069002B0526052B07400AB70C89009C
:1000700043073C0A1B0C88000307400A2B04260494
:100080000607440A0B05450A0B0403092E06500A0D
:100090000E065A0A07075A0A6C006D002E0506055F
:1000A0001E0C8D004307560A840C8C0003075A0A65
:1000B0002E04060407075E0A0E055F0A0E040309F4
:1000C0002606660A6F0070002704710A2706710A67
:1000D000980C90000307710A960C8F000307710AB1
:1000E000270503094706780A2707790A4605790A8A
:1000F000460403094606800A7100720047048B0A11
:1001000047068B0A4C0C920003078B0A4B0C91009C
:0A01100003078B0A47050309240AC0
:0203FE00000CF1
:080400000000010000000000F3
:021FFE00FA0FD8
:00000001FF
